:020000040000FA
:060000000219FD0200B32D
:03002B0002008D43
:03005B0002028C12
:030073000200A0E8
:100080000406080C10182030406080A0C0C0D0C00A
:10009000E0C2CF0541E52360021523D0E0D0D03285
:1000A000C2AF53E67F7592FA7593FFC22053917FDA
:1000B000D2AF32C2AF53E6EFC0D0C0E0C0F0D2D36F
:1000C000D2AF5388EFA88AA98C758A00758C00433B
:1000D000881030331FE8C4540FFAE9C454F04AFAC8
:1000E000C3132AFAC3E833F8E933F9E82AFAE93402
:1000F00003FB213D30320FC3E833E933FAE82AFA33
:10010000E93400FB213D303115E875F056A4AAF022
:10011000E975F056A42AFAC5F03400FB213DE875D4
:10012000F02BA4AAF0E975F02BA42AFAC5F034004C
:10013000C313FBEA13FAC3EB13FBEA13FAC3EB9402
:10014000095006C3EB9403501A0522E522700215EC
:1001500022C3E522940A5002417F7552007A007B47
:1001600000414DE522600215223035067C007D04F9
:10017000217DAC31AD32303A04AC33AD34C3EA9CAE
:10018000FAEB9DFB9208AE5EAF5F303A425007201B
:100190003409D234219B303402C234303404AE608E
:1001A000AF61203902B234C3EA33FAEB33FBA20861
:1001B000500AEAF42401FAEBF43400FBC3EA942871
:1001C000FAEB9400FB501478007A007B0021DBA24C
:1001D00008500878007A007B004131E5255403601F
:1001E00019202A16E55BF9EB7007C3E99A4002E98A
:1001F000FAE53CC42AFAEB3400FBEA8EF0A4F9AA33
:10020000F0EB8EF0A42AFAC5F03400FBC3EB13FD2B
:10021000EA13F80FEF146004C3E833F8C3E933EAD4
:1002200033FAEB33FBDFEDEB30E20678FF7AFF7B4E
:10023000038852D230C3E559FC955A4002AC5AC3E8
:10024000EC95525008EC75F004A4FAABF0EAF4F81F
:10025000EBF45403F9C3E89428FAE99400FB500442
:100260007A007B00885489558A568B5775230AD0AB
:10027000F0D0E0D0D053F7DF43F74043E6103275BB
:10028000230AD0F0D0E0D0D043E61032C2AF53A85A
:10029000FEC0D0C0E0D2D3A8F9E55830E10AE5FAB3
:1002A00020E14220E03F41B0E5FA30E13820E0357E
:1002B000C3E55513F8E55413F5FB88FCC3E5571364
:1002C000F8E55613F5E988EA85555853F7BFC3E5B5
:1002D000529401400575530041E5E5532401F5535F
:1002E00050037553FF53F7DFD0E0D0D043A801D2BD
:1002F000AF327901801479038010790A800C791E5D
:1003000080087964800479C880007817E4D5E0FD1E
:10031000D8FAD9F6227A147B7880127A107B8C80F6
:100320000C7A0D7BB480067A0B7BC88000E562D521
:10033000E001227902E4D293D5E0FDD292D5E0FD2E
:10034000C292D5E0FDC293D5E0FDE920E002D29053
:1003500030E002D294E562D5E0FDE920E002C290EF
:1003600030E002C2947496D5E0FDD9C9EAF8D5E030
:10037000FDD8FBDBB8D2932278FF20282879A1E7AB
:100380006023E548601F74FF8548F084853FF030A6
:10039000290375F005A4F8C5F0600278FFC3E8955D
:1003A0005B5002A85B885A22C3E54794E4E5489471
:1003B00000E55A50031461B9046002F55A2275E849
:1003C0009022055CC3E55C9408405330EDF4A8BD71
:1003D000A9BE755C00E9FA79A0E76041EA7006E51C
:1003E0005D6018800CC3E8955D600EE55D500560AA
:1003F0000A1480070460FA8002E55DF55DC3956725
:10040000401B7559C0C394044013755980C39404AC
:10041000400B755940C39404400375590022E559B7
:100420002410500274FFF55922743279A687F0A483
:10043000C5F0A2F733F8C3E895594002A859885B84
:10044000227547007548F022C2AF75C800A8CCA934
:10045000CDAA4130CF010A75C804D2AFAB42AC433C
:1004600088428943C3E89BF8E99C202808F9302C8E
:1004700002A15781B1AD448A44F9EA9DFA6004783B
:10048000FF79FFAE45AF468B458C46A842A943C3D2
:10049000E89EF8E99FF9C3E54813FBE54713FAE83E
:1004A0002AF547E93BF54850067547FF7548FF8137
:1004B000FEAA47AB48AC47AD487E047F02C3EB942D
:1004C00004400D1E1FC3EB940840052029021E1F87
:1004D000C3ED13FDEC13FCDEF7C3EA9CFAEB9DFBC6
:1004E000EF6009C3E913F9E813F8DFF7EA28FAEB3C
:1004F00039FB8A478B4850067BFF8B478B48C3EB01
:1005000094025002D22C3028047F03A1297892E66D
:10051000FFC3E53D948240110FC3E53D94A0400127
:100520000FC3EF940640027F057E02E548C4540FD6
:10053000F9E548C454F0F8E547C4540F28F8C3E877
:100540009EFAE99400FB4009C3EA9401EB94005041
:10055000047A01E4FBA1A3AA47AB48EBC4FEEAC4BA
:10056000540F4EFCC3EA9CFAEB9400FBC3E813C3A0
:1005700013F8EA28FAEB3400FB8A478B48C3EB9464
:10058000024002C22C7802EBC4FE7B00EAC4540F86
:100590004EFAC3EA98FA4005C3940150027A0178F2
:1005A00092E6FF302002A1A3854E92854F93D22080
:1005B00043E680C3E49AF8E49BF9302C02C12EE8AC
:1005C000FAE9FBD3E913FDE813FC884E894FC3EF2A
:1005D00094036037EF20E00CE82CF8E93DF9ECFAE1
:1005E000EDFB8013E828F8E939F9C3E82401F8E9BC
:1005F0003400F97AFF7BFFC3EF9403400E8A508BDF
:1006000051884A894B8C4C8D4DC162885089518AE2
:100610004A8B4B8C4C8D4D3028127550F07551FF24
:10062000754CF0754DFF754EF0754FFFC162E8FADD
:10063000D3E813FC884EC3EF94036020EF20E0075B
:10064000E82CF8ECFAC14EE8282401F87AFFC3EF51
:10065000940340088A50884A8C4CC16288508A4A68
:100660008C4C302002C162753A02D22043E680E50C
:100670002554036034A847A948C3E913F9E813F8DF
:10068000C3E913F9E813F8302804E92440F9C2AFAC
:1006900053E67F759100C3E498F594E499F5957558
:1006A0009104D22043E680D2AF22D2217549007551
:1006B0002000302B03752040800ED2217549007533
:1006C0002040302B0375200078017901202C20E593
:1006D0002554036002C2217914E548C31370010454
:1006E000F8C3941440027814302804781B791B2036
:1006F0002010E549600C302803D53A04D223E1727A
:10070000D16A0549E59B5440B52002E15C302809D7
:1007100008C3E899400118C1EF20210A08C3E899ED
:100720004002C1C8C1EFC221C2AF53E67F7591003C
:10073000302C127594007595F8759104D22043E61B
:1007400080D2AFC1C8E5487EFFC3334005C3334004
:1007500001FEC3E49E759400F595E139C3E5399433
:10076000015002C1C8302102C1C8D802E170C1EFF6
:10077000C223C2AF53E67F75910085509485519591
:10078000759104854A92854B93D22043E680D2AF7F
:10079000E525540360072029020539801030230D18
:1007A000202B0A20210715811581020E8B2278004B
:1007B0003021027801E53D75F007A4F9E5F028F550
:1007C000F0E9A2F013A2F113A2F213F53DC394785D
:1007D0005003753D78C3E53D953E400BD222C29053
:1007E000C292C29475D53F302002E1E7854C9285D4
:1007F0004D93D22043E68022203810C2AFD293C25C
:100800009175D50FD2AF759F0301CCC2AFD293C201
:100810009575D53CD2AF759F0301CC203811C2AF7E
:10082000C29475D533C291D2AF759F130208CCC262
:10083000AFC29075D533C295D2AF759F230208CC55
:10084000203810C2AFD291C29575D533D2AF759F03
:10085000238079C2AFD295C29175D533D2AF759F3F
:10086000138069203811C2AFC29275D53CC295D2AF
:10087000AF759F030208CCC2AFC29275D50FC2916B
:10088000D2AF759F030208CC203810C2AFD295C2F8
:100890009375D53CD2AF759F138031C2AFD291C250
:1008A0009375D50FD2AF759F238021203810C2AF2A
:1008B000C29075D50FC293D2AF759F23800EC2AF81
:1008C000C29475D53CC293D2AF759F13C22222C287
:1008D00090C292C294D291D293D29575D53F22788C
:1008E0008076FF0876FF0876FF0876FF0876FF0817
:1008F00076FF0876090876FF087601788C7601087D
:1009000076FF0876FF0876FF0876FF0876FF087600
:10091000030876FF0876FF0876FF0876250876D06C
:100920000876280876500876040876FF08760208CC
:1009300076FF08767A0876FF08760708760108764B
:10094000FF0876FF08760008760022FA75F00CA4FE
:10095000ABF0EAC333F8740133F9E8C333F8E93391
:10096000F9E8C32BF8E93400F9227888E6C3940348
:10097000D23A5002C23AC238E630E102D238A23846
:1009800092397886E6149000809378A6F67886E609
:10099000F53FC394025003753F02789CE6753EFF15
:1009A000B40203753EA0B40303753E8278A0E6F856
:1009B000600674282409D8FCF5677896E6314B88E0
:1009C000318932789EE6314B883389347897E63125
:1009D0004B8835893611CF223035117A007B007C67
:1009E000FF7D007E00513F8B5F8A5E22303A227885
:1009F00096E6FA7B00789EE6FC7D00C3EA33FAEBCC
:100A000033FBC3EC33FCED33FD7E0A513F8B618A2F
:100A1000607896303A02789EE6FA7B007897E6FC9A
:100A20007D007E00303A10C3EA33FAEB33FBC3ECAF
:100A300033FCED33FD7E0A513F8B5F8A5E2222C379
:100A4000EC9EFCED9400FDC3EC9AFCED9BFDC3EC29
:100A50009423ED940050047C237D00C3EC94FFEDBF
:100A6000940140047CFF7D017BFF0B7A000AEA7051
:100A700009C3EC33FCED33FD416AEC8AF0A4AEF01F
:100A8000ED8AF0A42E947C40E4EAF460DD22D235B5
:100A900031D81202FE1202FE7A007B007C10120294
:100AA000F6E5522AFA74003BFBDCF37C04C3EB133B
:100AB000FBEA13FADCF7FFEB60027FFFC23531D8A7
:100AC0002278A5E6F954037000E9540C7000E9544B
:100AD000307000E954C070002275650075660075BD
:100AE00097DE7597AD7581C043FF8075EF0675A9D8
:100AF0000011CF7580FF75F1F075A4007580FF754A
:100B0000D4FF75902A75F23F75A53F75902A75D56B
:100B10003F75A60175E34075E20211CFE4F8F6D8FF
:100B2000FD11DFD1BD78988662753001C2AF120326
:100B3000061203151202FE12031B1202FE120321FB
:100B40001202FE51C1C2AF75650075660078FA7970
:100B5000FA308507D9FBD8F7021C00316A31D87802
:100B600098866211CF75E405758811758E047589B4
:100B70000975C80475910475D84075D90875F78151
:100B8000759E0375960075DA4275DB4275A821756E
:100B9000E69075F310759B80759D0075D10C75BC42
:100BA0005975BB1075E88075B2011202F2D2AF75AB
:100BB0003C00C230120306C231752200120302C388
:100BC000E522940A4024D231C23275220012030277
:100BD000C3E522940A4013D232C2337522001203B5
:100BE00002C3E522940A4002D2331202F6203003F7
:100BF000020B45C2AF120315120315120315D2AF33
:100C0000120306303A0281A61202F6788CE6C394EB
:100C100001500281A6E530C39401500281A675659A
:100C2000A57566F17F02D23531D8120302C2AFC278
:100C30003531D8C3E552947FD2AF406A1202F2C276
:100C4000AF120327D2AFDFDE518EC3EF7897F612D3
:100C50000306F19D7F0AD23531D8120302C2AFC21A
:100C60003531D8C3E552947FD2AF50E81202F2C2B8
:100C7000AF1203151202FA120315D2AFDFD8518E4C
:100C8000EF24037896F6F87997E7C3942340039806
:100C90005006E824237897F6120306D1F7F1CC1218
:100CA000030231D86145756500756600120302784C
:100CB00001303A027805C3E5529840028103C2AF81
:100CC000120327120327120327D2AF12030675302F
:100CD00000E4F537F5380537E537F4703E05387828
:100CE0009AE67819146012783214600D787D1460D9
:100CF0000878FA146003753800C3E53898401C1171
:100D0000CF1202F2153875370078998662C2AF1299
:100D10000327D2AF789886621203021202FAE52303
:100D2000700261457801C3E5529840AA120302E5BA
:100D3000237003020B45C2AF11CFE4D2AFE4F55CE0
:100D4000F524F525F53D755C081202F21203BE305C
:100D5000EDFDA8BDA9BEE97001F8885D1203C2755A
:100D60005C08C2AF7559FF120429855B59855B5A2F
:100D7000D2AF303A07C238303402D238D22875396F
:100D800000118811AB1204411204481204411204EC
:100D9000481204411206BA1207AE1207F8120448AC
:100DA0001206AA202C03120378302C031203A81277
:100DB00007AE111B1204481206BA1207AE114012F8
:100DC00004481206AA1207AE11631204481206BAAA
:100DD0001207AE11881204481203BE1206AA1207A7
:100DE000AE11AB1203C2120448302827855B597933
:100DF000187A0CC3E53999400EC228D2298A3B855E
:100E00005B59855B5A800CC3E55294014003020D87
:100E100094C19330291C202B19E53B147006C2297C
:100E2000D22AA194F53BC3E55294014003020D94EC
:100E30008061753C0078FA79A4E760027803C3E525
:100E40005398504FE523604B303A17203805203433
:100E500007800F303402800A202B07D22B855B5984
:100E6000A1C278F0302B05855B597820C3E54898FE
:100E70005003020D94302B1BC22BC238303402D2E7
:100E800038D229753B12855B59A194053CE5526027
:100E900002C196753C00C2AF11CF752400752500C4
:100EA000D2AF12030211CF78A4E66006C291C293BA
:100EB000C295C3E53C94044002614581D1901A0D6E
:100EC0007820F130E520B4550AA3F130E520B4AA2A
:100ED00002800611DFD1F7801D901A0378807B0A0B
:100EE000F130A308DBFA901A0F788C7B1AF130A34B
:100EF00008DBFA901A2922C2AFF173F150901A0060
:100F00007410F135A37403F135A37421F135901AEF
:100F10000378807B0AF134A308DBFA901A0F788CEF
:100F20007B1AF134A308DBFAF186F164901A2922C6
:100F3000E493F622E6438F01538FFDFFC3E58394CC
:100F40001C400122EF8565B78566B7F0538FFE22FE
:100F5000438F02438F018565B78566B7901A0DF000
:100F6000538FFC22901A0D7455F135901A0E74AA05
:100F7000F135227A3079D07820901A40F130E5208E
:100F8000F709A3DAF7227A3079D0901A40E7F135E1
:100F900009A3DAF9227C05120306DCFB22C2AF1298
:100FA000031512031B1203211203271202FA120364
:100FB0001512031B1203211203271202FA12031542
:100FC00012031B120321120327D2AF22C2AF120356
:100FD0002712032112031B1203151202FA12032710
:100FE00012032112031B1203151202FA1203271215
:0B0FF000032112031B120315D2AF22D5
:1019FD00020AD9100321FFFFFFFFFFFF09FF01FFBF
:101A0D0055AA01FFFFFFFFFF03FFFFFF25D0285061
:0D1A1D0004FF02FF7AFF0701FFFF0000FF3A
:101A400023445F4C5F34302320202020202020209E
:101A500023424C48454C492445464D3842313023B9
:101A60002020202020202020202020202020202076
:101C0000C2AFC2D37597DE7597AD7581C075A90057
:101C100043FF80752438752503B1DB7529A5752A26
:101C2000F143F12053A4DFD28575D4FF75E3407DE5
:101C3000FA780379E67C10752200752300901DE880
:101C40007B0675249875250130850281482085081A
:101C5000D8FBD9F9DCF781BA308508D8FBD9F9DC93
:101C6000F781BAB19BE493A3C39A6004DDC381BA40
:101C7000DBDBB18D600281317B08E493FAA3B16EA6
:101C8000DBF87A30B16E752200752300B18DEAFC65
:101C9000EBFDC3ED94FE400EB18D8A278B28ED300D
:101CA000E0048A828B83B18D7AC270D8C3ED94FE32
:101CB000601950CEBD0029EC600F7520007521FF22
:101CC000752900752A000200008100A827A92808AC
:101CD00009D804D90281DDB191EAF281D10D81A642
:101CE000C3ED94035051EDA2E092007AC5C3E582A2
:101CF0009400E583941C508C200010438F02438F86
:101D0000018529B7852AB7F0300027A827A9280818
:101D100009438F01538FFDD804D902A132C3E58353
:101D2000941C4003A3A117E28529B7852AB7F0A325
:101D3000A117538FFC81827AC1BD030CE493A3FAEF
:101D4000B152DCF8B14A81828184AA22AB23B16E00
:101D5000EBFAEA6222752608C3E52313F523E52290
:101D600013F52250066323A0632201D526EAB1DBD6
:101D7000B1DB75260AEAF4200102D285300102C2E5
:101D800085B1DBC3134002C201D526EB22B191EA33
:101D9000FB208502A191308502A196752608AE240C
:101DA000AF25C3EF13FFEE13FEB1DFB1DBC3EA13C0
:101DB0003085024480FA30E703632201C3E5231330
:101DC000F523E52213F52250066323A0632201D5F3
:101DD00026D9E52265236523F52222AE24AF250E00
:101DE0000FDEFEDFFCD20122424C48656C693437BD
:061DF0003163E8B10601B9
:00000001FF
